:100000003EC1000058C1000056C1000054C10000AC
:1000100052C1000050C100004EC100004CC10000A0
:100020004AC1000048C1000046C100000C94A60B64
:1000300042C1000040C100003EC100003CC10000C0
:100040003AC1000038C1000036C1000034C10000D0
:1000500032C1000030C100002EC100002CC10000E0
:100060002AC1000028C1000026C1000024C10000F0
:1000700022C10000EF02F402FF0209030F0315037F
:1000800042034E035303580367036C037703930340
:10009000A603AC03B403BA03C003CA031A043A04A8
:1000A00050045F0461055D056505690563055F052D
:1000B00067056B05730C960C810D960C810DDD0C9C
:1000C000FF0C810D520D640D2203690062006D006A
:1000D0002D00630061007000730065006E00730006
:1000E00065002D00750073006200000022035400BB
:1000F0006F006D00200057006F006E0067002D003C
:1001000043006F0072006E0061006C006C00000024
:100110000403090409025400030100A03209040089
:10012000000103010100092111010001222500073E
:1001300005810308000A0904010001030000000909
:1001400021110100012220000705830308000A098C
:10015000040200010300000009211101000122BE78
:10016000000705820319000A120110010000002097
:10017000810402000100010200010600FF0901A143
:10018000010902150025FF7508950881020903156C
:100190000025FF750895089102C005010906A10117
:1001A0000508190129031500250195037501910220
:1001B000950175059101050719E029E7150025014D
:1001C00095087501810205071900293115002501DF
:1001D0009532750181029501750181010507193379
:1001E000299B15002501956975018102950175010D
:1001F00081010507199D29A41500250195087501A0
:1002000081020501198129831500250195037501D6
:100210008102050C19B029B8150025019509750151
:100220008102050C09CD09E209E909EA0A8A010AF5
:1002300092010A94010A21020A23020A24020A25D1
:10024000020A27020A2A0215002501950D7501816F
:1002500002950175028101C005010906A101750120
:100260009508810195017508810195057501910138
:10027000950175039101950675088101C00011244F
:100280001FBECFEFD4E0DEBFCDBF11E0A0E0B1E0F4
:10029000EEE5F0E202C005900D92A635B107D9F760
:1002A00013E0A6E5B1E001C01D92A837B107E1F760
:1002B0008FD00C942D10A4CE1DC313C380E291E007
:1002C0000E94EA0E80E191E00E94EA0E80E091E057
:1002D0000E94EA0EE2EEF0E080818460808308955F
:1002E00080E291E00E94B40D80E191E00E94B40DA3
:1002F00080E091E00C94B40D80912E0190912F013B
:10030000009729F0019790932F0180932E018091FF
:100310001E0190911F01009729F0019790931F01F2
:1003200080931E0180910E0190910F01009729F09A
:10033000019790930F0180930E01E3C20F931F93D7
:10034000CF93DF93FC01C901E80121E0E032F2071D
:1003500011F44CD305C021E0E031F20721F4CCD1F7
:1003600088E090E005C066817781D1D389E190E093
:100370009983888380E0DF91CF911F910F91089539
:10038000AC01C90121E04032520709F48DC440514B
:10039000514009F417C18BC484B7877F84BF88E1BB
:1003A0000FB6F89480936000109260000FBE90E04A
:1003B00080E80FB6F89480936100909361000FBEBF
:1003C0003AD046D789D249D7479A47980C94970B89
:1003D000E3DF7894FCD21CD690D6E1D28FE19EE484
:1003E0000197F1F700C0000049D0809184019091FD
:1003F0008501019609F41BD55DD480916F03882394
:1004000021F080916F03853039F480916D0388234A
:1004100019F0D4D5811137D780E291E00E94FD0E0A
:1004200080E191E00E94FD0E80E091E00E94FD0ECF
:100430000E949A0DE1CFFDD6289A0895CF93DF93BD
:1004400090938501809384012898EC01CC0FDD1FE7
:10045000CC0FDD1F8D2FF6D68C2FF4D6289ADF9186
:10046000CF9108956091840180E090E00E941B107C
:100470006091850181E090E00C941B10CF93DF9395
:1004800081E090E00E940410C82FD0E0DC2FCC2740
:1004900080E090E00E9404109E01282BC901DF91AA
:1004A000CF91CCCF292F332723303105C9F064F405
:1004B0002130310581F02230310509F043C084E557
:1004C00090E024E131E042C021323105F1F02232E6
:1004D000310541F137C082E190E028E631E036C0D5
:1004E00099278130910541F08230910541F0892BA7
:1004F00049F5E0E1F1E005C0ECEEF0E002C0E8EC27
:10050000F0E0849190E09F0121C06330D8F4E62FA1
:10051000F0E0EE0FFF1FE25CFE4F2081318189E0A9
:1005200090E014C0633070F470E0FB01EE0FFF1F29
:10053000E85CFE4F20813181FB01EB5CFE4F808146
:1005400090E004C080E090E020E030E0FA013183E8
:1005500020830895EF92FF920F931F93CF93DF9321
:100560008C0191E0EE24E394F12C461720F1A62FA4
:10057000B0E0AA0FBB1FAA0FBB1F20E030E0E801CC
:10058000C90FD11DF901EA0FFB1FE757FE4F80810C
:1005900083304CF08881F701022E01C0EE0F0A94DF
:1005A000EAF7E82BE8832F5F3F4F2430310551F7FE
:1005B0006F5F9F5FDACFDF91CF911F910F91FF9017
:1005C000EF900895DC01EC914E2F50E04D30510535
:1005D00008F091C0FA01E65CFF4F0C94D10F119620
:1005E0008C9180933201089511962C911197129657
:1005F0008C9190E0982F8827820F911D1FCF119624
:100600008C91882309F477C0E0913301F091340193
:10061000099411968C91882309F46DC023CF11960B
:100620008C91882309F467C002C413964C911397E8
:1006300012969C9112971196EC918E2F8F738731A1
:1006400008F059C0943008F056C0E295E695E6955A
:10065000E370E150E33040F4F0E0EE0FFF1FEC5B9D
:10066000FE4F2081318102C020E532E0E82FF0E02A
:10067000EE0FFF1FEE0FFF1FE90FF11DE20FF31F3B
:100680004083089512968C9112971196EC91E83060
:1006900090F5F0E0E85FFC4F8083089511968C910F
:1006A000882349F12AC511968C91882321F140C5F0
:1006B00013968C91139712969C91129711962C91E8
:1006C00020938701909386018093880113C111962E
:1006D0008C91882381F051C111968D919D91AC919F
:1006E0008093E5019093E601A093E70108951196A8
:1006F0008C91811185C40895CF93DF93DC0188E04C
:10070000FD0111928A95E9F7E0913201EC934E2FA9
:1007100050E0FA013197EB30F10508F0DAC0E95BFF
:10072000FF4F0C94D10F84E011968C93119798E0B1
:1007300012969C93129797E113969C931397149695
:100740008C93149781E015968C93C3C046E060E0CB
:10075000CD0100DF83E005C04DE067E0CD01FADEAA
:1007600084E080933201B5C044E16EE0CD01F2DE59
:1007700085E0F7CF47E165E1CD01ECDE82E0F1CF26
:10078000909184018091850111969C931197129606
:100790008C939FC08091810190918001282F229598
:1007A000220F220F207C292B11962C931197C09198
:1007B0003001D09131011296492F50E0440F551F5E
:1007C000440F551F20E030E0F901E40FF51FEC0F56
:1007D000FD1F60816D932F5F3F4F24303105A1F7DE
:1007E0009F5F973119F09093800173C01092800140
:1007F0008F5F843019F08093810102C010928101D3
:1008000080918101813061F040F0823081F083304D
:1008100009F05FC08CEA92E005C080E592E002C07A
:1008200080E193E0909331018093300152C084EFD6
:1008300091E0F8CF80917F0111968C931197E82F6A
:10084000F0E0EE0FFF1FEE0FFF1FE85FFC4F40814F
:1008500051816281738112964D935D936D937C9368
:1008600015978F5F823019F080937F0132C010920C
:100870007F012FC0E0E5F1E080E090E022E0280F6A
:1008800031910196ED01C80FD91F3883332321F030
:100890008630910599F727E0A20FB11D1C9219C06F
:1008A0008091870111968C93119780918601129601
:1008B0008C9312978091880113968C930AC0209193
:1008C000E5013091E6014091E70111962D933D93AA
:1008D0004C93DF91CF910895249A259A269A279ACE
:1008E00008952C982D982E982F981092830110928D
:1008F00082010895F6DF80918701813009F42F9AF3
:100900000895809183018F3F19F08F5F8093830159
:10091000809187018130B1F49091830180918601AB
:10092000981302C02E98089580918201882351F077
:1009300020918801921730F01092830181508093AA
:1009400082012E9A0895809182018F5F80938201A7
:10095000089590918701923079F480FF02C02D9A1A
:1009600001C02D9881FF02C02E9A01C02E9882FFEF
:1009700002C02C9A08952C980895609187018AE707
:1009800091E00E941B10609186018BE791E00E942C
:100990001B10609188018CE791E00C941B108AE792
:1009A00091E00E940410833018F48093870102C004
:1009B000109287018BE791E00E94041080938601DA
:1009C0008CE791E00E9404108093880108958CE5E3
:1009D000E9E8F1E0DF011D928A95E9F78CE0E8EEA5
:1009E000F1E0DF011D928A95E9F70895AF92BF9279
:1009F000CF92DF92EF92FF920F931F93CF93DF93EB
:100A0000EC01B1D38150833048F4E82FF0E0EE0FD1
:100A1000FF1FE65BFE4F4081518102C040E552E07E
:100A200060E070E0D12CEE24E394F12CFD2D20E069
:100A300030E08B011595079508511E4F862F817068
:100A4000C82E95E0B92EBD1408F44EC0D8018C9183
:100A500090E0CC2051F0D9011496570102C0AA0CA5
:100A6000BB1CAA95E2F7D50107C0D701022E02C030
:100A7000AA0FBB1F0A94E2F78A239B23892B69F1F3
:100A8000DA01A20FB31FEC91E43038F180E38E0F4E
:100A9000833018F1D394DE01AF0FB11D1296EC93A1
:100AA0008E2F90E0FC01E05EF109E830F105A8F43A
:100AB000EE5AFF4F88810C94D10F8E5F0DC0805E7F
:100AC0000BC08F5F09C0805F07C08C5F05C0805C72
:100AD00003C0885F01C0805888832F5F3F4F243058
:100AE000310511F0FD2DADCF6F5F7F4F4C5F5F4F34
:100AF0006731710509F09ACFDF91CF911F910F9166
:100B0000FF90EF90DF90CF90BF90AF9008952F921D
:100B10003F924F925F926F927F928F929F92AF928D
:100B2000BF92CF92DF92EF92FF920F931F93CF93DA
:100B3000DF938C014B0117D38150833048F4E82FA9
:100B4000F0E0EE0FFF1FE65BFE4F8081918102C057
:100B500080E592E06C01212C312C66246394712C89
:100B6000412C512CC10195958795FC01E851FE4F10
:100B70005F01D22DD170F501808190E0DD2359F025
:100B800092012C5F3F4FA30102C0440F551F2A95CD
:100B9000E2F79A0107C09301042C02C0220F331F11
:100BA0000A94E2F782239323892B09F450C0F601BB
:100BB000E40DF51DC081C13E99F060F4C33D38F4E9
:100BC000C03D08F044C0C33008F441C021C0C03E5D
:100BD00099F01EC0C53E21F078F0C83EC8F40CC0A4
:100BE000F401808190E020E22C0F02C0959587955A
:100BF0002A95E2F780FFA7DEC05EC3010C2E01C07C
:100C0000880F0A94EAF7F8019081892B80831FC02E
:100C1000EC2EE694E694E694F12CC770F401EE0D08
:100C2000FF1D818190E00C2E02C0959587950A9456
:100C3000E2F780FF88DEF801EE0DFF1DC3010C2EE8
:100C400001C0880F0A94EAF79181892B8183FFEF15
:100C50004F1A5F0A24E04216510409F08CCF3FEF8F
:100C6000231A330A44E0C40ED11C57E1251631047F
:100C700009F076CFF8018181887F8183838D887F19
:100C8000838FDF91CF911F910F91FF90EF90DF90B5
:100C9000CF90BF90AF909F908F907F906F905F901C
:100CA0004F903F902F900895FC01808152CEFC011F
:100CB00080814FCE4F925F927F928F929F92AF92A0
:100CC000BF92CF92DF92EF92FF920F931F93CF9339
:100CD000DF9300D000D0CDB7DEB78CE0E8EEF1E0D6
:100CE000DF011D928A95E9F779E8E72E71E0F72E8A
:100CF00000E010E0AA24A394E5E0BE2EDD24D39406
:100D0000F8ECCF2E902EE02FE695E695E695F0E0F4
:100D1000EB51FE4F808190E0202F277002C0959507
:100D200087952A95E2F780FD65C0802F9ED2479A6D
:100D3000479819821A821B821C828A2D8A95F1F7A4
:100D40004899A9824999AA824A99AB824B99AC8267
:100D5000AE014F5F5F4F2701D70120E030E0C801AF
:100D60009595879588519E4FE92DE1709E2E722EA4
:100D7000FA016191AF01F201662319F060816150BF
:100D800002C060816F5F6083BD018C9087FE02C0EE
:100D90001C9204C0F5E0F8150CF4BC921196FB010E
:100DA00060816330B4F0FC018080992051F0B9017A
:100DB0006C5F7F4FFD2D01C0FF0F6A95EAF76F2F23
:100DC00005C06D2D01C0660F7A94EAF76829FC0111
:100DD00060832F5F3F4FFFEF4F1A5F0A24303105CA
:100DE00031F63BD2479A47980631110519F08C2D00
:100DF0008A95F1F70F5F1F4F64E0E60EF11C073193
:100E0000110509F07FCF0F900F900F900F90DF9199
:100E1000CF911F910F91FF90EF90DF90CF90BF90F7
:100E2000AF909F908F907F905F904F900895AF927A
:100E3000BF92CF92DF92EF92FF920F931F93CF93C7
:100E4000DF9340E552E027E1B12CD12C80E090E027
:100E5000FA01E80FF91F3081313021F0323019F4F6
:100E6000D39401C0B39401968430910589F7215041
:100E70004C5F5F4F2111EACFC0E0D0E00FEF13E0ED
:100E8000E12CF12CC8018E199F0982309105C0F127
:100E9000EC01D695C795CE0DDF1DCE01CFDA8FE8D8
:100EA00091E00197F1F700C0000070E2C72E02DF69
:100EB000CA94E9F729E831E060E572E040E080E0BB
:100EC00090E0F901E80FF91F508153303CF0FB012D
:100ED000E80FF91F5081543008F04F5F01968430BD
:100EE000910579F72C5F3F4F6C5F7F4F91E0253E76
:100EF000390729F74D1510F08E01C4CF7E01C2CFFE
:100F00008E01EE24EA9453E0F52EC12CD12C9701EA
:100F10002C193D0922303105C0F1E901D695C7955C
:100F2000CC0DDD1DCE018ADA8FE891E00197F1F753
:100F300000C0000040E2A42EBDDEAA94E9F789E8D3
:100F400091E060E572E040E020E030E0FC01E20F7B
:100F5000F31F508153303CF0FB01E20FF31F50812F
:100F6000513009F44F5F2F5F3F4F2430310571F747
:100F700004966C5F7F4F21E0853E920729F74B1561
:100F800010F07E01C4CF6E01C2CFC8018C1B9D0B37
:100F900024E0969587952A95E1F76FE070E0F0D709
:100FA0008C0F9D1F4BDADF91CF911F910F91FF9016
:100FB000EF90DF90CF90BF90AF909CCC20E532E0D7
:100FC00049E851E080E090E0FA01E80FF91F608104
:100FD000633034F0F901E80FF91F6081643070F478
:100FE00001968430910581F72C5F3F4F4C5F5F4F36
:100FF00082E02C3A380731F780E0089581E00895C7
:1010000043E050E06DE771E085EE91E00C940C1048
:1010100043E050E06DE771E085EE91E0E5D7809127
:10102000E5018F3F71F48091E6018F3F51F480918B
:10103000E7018F3F31F41092E5011092E601109222
:10104000E7010895AF92BF92CF92DF92EF92FF92A5
:101050000F931F93CF93DF93EB015C012CE5A20E5E
:10106000B11C6C01F4E0CF0ED11C7E018C010F5F2E
:101070001F4FCAD78F3F09F480E0F70181937F01AA
:10108000C8010C151D0591F724960A151B0549F793
:10109000DF91CF911F910F91FF90EF90DF90CF9054
:1010A000BF90AF900895AF92BF92CF92DF92FF9220
:1010B0000F931F93CF93DF938C01EB0187E1F82E01
:1010C0006E0184E0C80ED11CC80169915C012FEF4C
:1010D000A21AB20AB0D7C501CC15DD05B1F70C5F75
:1010E0001F4FFA9469F7DF91CF911F910F91FF90F5
:1010F000DF90CF90BF90AF90089548E050E062E756
:1011000071E088E093E070D760E572E082E090E003
:1011100099DF60E173E08EE590E094DF64EF71E0C9
:101120008AEB90E08FDF6CEA72E086E191E08ACF93
:1011300048E050E062E771E088E093E06DD760E559
:1011400072E082E090E0AFDF60E173E08EE590E076
:10115000AADF64EF71E08AEB90E0A5DF6CEA72E051
:1011600086E191E0A0CFCF92DF92EF92FF921F93A2
:10117000CF93DF93A0E5B2E040E050E090E0C1E023
:10118000D0E0FA01F595E795E851FE4FE081CE2ECB
:10119000D12C20E030E0142F1170112359F0B90147
:1011A0006C5F7F4F7E0102C0EE0CFF1C6A95E2F778
:1011B000B70107C0BE01022E02C0660F771F0A9456
:1011C000E2F76C217D21672B81F0BD01620F731F57
:1011D000FB018081813D31F0823D31F0803D29F479
:1011E000916003C0926001C094602F5F3F4F243034
:1011F000310599F64F5F5F4F14964731510509F657
:10120000992371F0E8E0F3E028E02E0F8191382F68
:1012100032953F70391302C08F7003C02E13F6CF82
:1012200080E0DF91CF911F91FF90EF90DF90CF9002
:101230000895219A209A229A84E58CBD8DB581600B
:101240008DBD08958EBD0DB407FEFDCF8EB50895FA
:101250003C9A3D9A3E9A3F9A08954598449888E171
:10126000459A45988150E1F7089545984498449AE5
:10127000459A4598449890E0981721F0459A4598EA
:101280009F5FFACF089584E089BD86E089BD09B4E7
:1012900000FEFDCF8091D8008F7D8093D800809193
:1012A000E00082608093E0008091E00081FDFCCF4F
:1012B0000895CF92DF92EF92FF920F931F93CF93F7
:1012C000DF93EC018B017A01C9D1811133C0E114A4
:1012D000F10439F0F70180819181081B190BC80FC7
:1012E000D91FC12CD12C0115110519F18091E800ED
:1012F00085FD16C08091E8008E778093E8001AD4AF
:10130000E114F10449F0F70180819181C80ED91EE2
:10131000D182C08285E00EC0A1D1882321F30AC00A
:1013200089918093F10001501109FFEFCF1ADF0A74
:10133000DACF80E0DF91CF911F910F91FF90EF9076
:10134000DF90CF9008952091760330917703261790
:10135000370748F06115710539F42091E8002E77C0
:101360002093E80001C0B90140E06115710581F1E9
:1013700020916F032223E9F12530E9F12091E80063
:1013800023FD35C02091E80022FD2BC02091E8000C
:1013900020FFEBCF2091F20030E0FC01CF0161157E
:1013A000710559F02032310540F481918093F100AC
:1013B000615071092F5F3F4FF1CF41E0203231057D
:1013C00009F040E02091E8002E772093E800CDCF8F
:1013D0004111CECF06C080916F03882351F0853034
:1013E00051F08091E80082FFF6CF80E0089581E01F
:1013F000089582E0089583E008956115710529F448
:101400002091E8002B772093E800FC01611571051D
:1014100021F180916F03882341F1853041F1809162
:10142000E80083FD20C08091E80082FFEFCF80912B
:10143000F200882331F08091F100819361507109AD
:10144000B1F78091E8008B778093E800DFCF80913F
:101450006F03882351F0853051F08091E80080FFC0
:10146000F6CF80E0089581E0089582E0089583E05A
:10147000089520917603309177032617370748F0B7
:101480006115710539F42091E8002E772093E8006A
:1014900001C0B901FC0120E06115710569F180917D
:1014A0006F038823D1F18530D1F18091E80083FD6D
:1014B00032C08091E80082FD28C08091E80080FF62
:1014C000EBCF8091F20090E06115710559F0803208
:1014D000910540F424912093F100319661507109F7
:1014E0000196F2CF21E0809709F020E08091E8009A
:1014F0008E778093E800D0CF2111D1CF06C08091A4
:101500006F03882351F0853051F08091E80082FF0D
:10151000F6CF80E0089581E0089582E0089583E0A9
:101520000895982F953058F59093E900981739F061
:101530007091EC002091ED005091F00003C0242F39
:10154000762F50E021FF19C03091EB003E7F3093A1
:10155000EB003091ED003D7F3093ED003091EB00DA
:1015600031603093EB007093EC002093ED005093CA
:10157000F0002091EE0027FF07C09F5FD3CF8F7050
:101580008093E90081E0089580E00895EF92FF9252
:101590000F931F93CF93DF93E62EEC018C010C5F2A
:1015A0001F4FF12CFE1499F19881992359F1F801FC
:1015B000208169817A8131973081892F8F708530C0
:1015C00010F080E025C0223010F442E001C046E077
:1015D000E8E0F0E020E0E617F70720F42F5FEE0FD9
:1015E000FF1FF9CF2295207F422B232F2295220F18
:1015F000220F207C991F9927991F622F692B91DF59
:101600008823F9F2F39425960B5F1F4FCBCF81E02F
:10161000DF91CF911F910F91FF90EF9008958091EE
:10162000700387FF11C08091E80082FD05C08091A2
:101630006F038111F8CF11C08091E8008B770BC048
:1016400080916F03882349F08091E80080FFF8CFF4
:101650008091E8008E778093E80008952091E4005F
:101660003091E50095E64091EC00842F817040FFB9
:1016700022C08091E80080FD1CC080916F03882308
:1016800091F0853091F08091EB0085FD10C0409184
:10169000E4005091E5004217530729F39A01915055
:1016A00011F784E0089582E0089583E0089581E0D1
:1016B000089580E008954091E80042FFDECF08954C
:1016C0003FD041D08091D8008F778093D80080910F
:1016D000D80080688093D8008091D8008F7D809357
:1016E000D80084E089BD86E089BD09B400FEFDCF45
:1016F00010926F0310926C0310926D0342E260E04F
:1017000080E00FDF8091E1008E7F8093E100809187
:10171000E20081608093E2008091E2008860809323
:10172000E2008091E0008E7F8093E0000895E3E680
:10173000F0E080818E7F808381E080936E03C0CF54
:101740001092E20008951092E10008951F920F9206
:101750000FB60F9211242F933F934F935F936F9384
:101760007F938F939F93AF93BF93EF93FF9380915A
:10177000E10082FF0BC08091E20082FF07C08091F0
:10178000E1008B7F8093E1000E947C018091E10069
:1017900080FF18C08091E20080FF14C08091E200B9
:1017A0008E7F8093E2008091E20080618093E2006E
:1017B0008091D80080628093D80019BC10926F038A
:1017C0000E945D018091E10084FF2EC08091E200C3
:1017D00084FF2AC084E089BD86E089BD09B400FE8B
:1017E000FDCF8091D8008F7D8093D8008091E1005B
:1017F0008F7E8093E1008091E2008F7E8093E200F3
:101800008091E20081608093E20080916C038111FD
:1018100006C08091E30087FD02C081E001C084E042
:1018200080936F030E945C018091E10083FF22C0DE
:101830008091E20083FF1EC08091E100877F80934A
:10184000E10082E080936F0310926C038091E100CD
:101850008E7F8093E1008091E2008E7F8093E20092
:101860008091E20080618093E20042E260E080E0EB
:1018700058DE5FD1FF91EF91BF91AF919F918F9112
:101880007F916F915F914F913F912F910F900FBE7C
:101890000F901F9018951F93CF93DF93CDB7DEB7AE
:1018A000AA970FB6F894DEBF0FBECDBFE0E7F3E016
:1018B00088E08E0F9091F10091938E13FBCF0E94E0
:1018C00070018091E80083FF1CC1809170039091AA
:1018D0007103492F50E04A30510508F012C1FA0156
:1018E000E65AFF4F5EC3803881F0823809F009C1A3
:1018F000809174038F708093E9008091EB0085FBE9
:10190000882780F91092E90007C080916D03882331
:1019100011F082E001C080E09091E800977F909301
:10192000E8008093F1001092F100C7C0282F2D7FAE
:1019300009F0E7C0882319F0823061F0E2C080919D
:101940007203813009F0DDC0933009F080E08093AC
:101950006D032DC080917203811129C080917403A1
:101960008F7009F4CEC08093E9009091EB0090FF56
:101970001EC090917103933021F48091EB0080623E
:1019800014C09091EB0090619093EB0021E030E067
:10199000A90102C0440F551F8A95E2F74093EA005F
:1019A0001092EA008091EB0088608093EB00109227
:1019B000E9008091E800877F83C08111A2C0109167
:1019C00072031F778091E3008078812B8093E3007E
:1019D0008091E800877F8093E80021DE8091E80015
:1019E00080FFFCCF8091E30080688093E3001111B9
:1019F00002C082E001C083E080936F0382C0805800
:101A0000823008F07EC080917203909173038C3D08
:101A100053E0950771F583E08A838AE289834FB7A3
:101A2000F894DE01139620E03EE051E2E32FF0E06F
:101A300050935700E49120FF03C0E295EF703F5FA1
:101A4000EF708E2F90E0EA3010F0C79601C0C0967C
:101A50008D939D932F5F243149F74FBF8091E8000C
:101A6000877F8093E8006AE270E0CE0101966BDC2C
:101A700013C0AE014F5F5F4F609174030E9452022A
:101A8000BC01009709F43DC09091E800977F9093C6
:101A9000E80089819A81EDDC8091E8008B77809362
:101AA000E8002FC0803869F58091E800877F809337
:101AB000E80080916C038093F1008091E8008E77BC
:101AC0008093E800ACDD1DC081111BC090917203B2
:101AD0009230B8F48091E800877F8093E80090937B
:101AE0006C039DDD80916C03811106C08091E30041
:101AF00087FD02C081E001C084E080936F030E94F3
:101B00005E018091E80083FF0AC08091E800877F32
:101B10008093E8008091EB0080628093EB00AA96AE
:101B20000FB6F894DEBF0FBECDBFDF91CF911F91EE
:101B300008950895CF9380916F03882399F0C09101
:101B4000E900CF709091EC00892F817090FD80E8C2
:101B5000C82B1092E9008091E80083FD9CDECF70D5
:101B6000C093E900CF9108956F927F928F929F92D8
:101B7000AF92BF92CF92DF92EF92FF920F931F939B
:101B8000CF93DF9300D01F92CDB7DEB77C01CDB6E7
:101B9000DEB68091E80083FF06C1F701808190E006
:101BA00020917403309175032817390709F0FBC0A1
:101BB00080917103833009F49DC030F4813071F05D
:101BC000823009F4D4C0EFC08A3009F4B8C08B3039
:101BD00009F4A1C0893009F0E6C04EC080917003BD
:101BE000813A09F0E0C08DB69EB61A8219828091C2
:101BF0007203109173038B83F7018085482F50E0A7
:101C00008DB79EB7841B950B0FB6F8949EBF0FBE81
:101C10008DBFEDB7FEB731965F0160E070E0CF0198
:101C2000DCD14FEF410F8E010F5F1F4F9501BE01B9
:101C30006D5F7F4FC7010E949E01F70186819781EA
:101C4000009721F0408550E0B501BED11092E90027
:101C50008091E800877F8093E80069817A81C501DF
:101C600072DB8091E8008B778093E8000FB6F894E0
:101C70009EBE0FBE8DBE97C080917003813209F069
:101C800092C0ADB6BEB60091760310917703709006
:101C90007203609073038DB79EB7801B910B0FB6D4
:101CA000F8949EBF0FBE8DBFEDB7FEB731964F01C2
:101CB0008091E800877F8093E800B801CF019DDB29
:101CC0008091E8008E778093E80021E0711001C0D8
:101CD00020E030E0021B130B280D391D4FEF460D9D
:101CE000672DC7010E94C0010FB6F894BEBE0FBE9B
:101CF000ADBE59C080917003813A09F054C0809103
:101D0000E800877F8093E8008091E80080FFFCCFA7
:101D1000F701818540C080917003813209F043C092
:101D20008091E800877F8093E80079DC90917203CE
:101D300081E0911101C080E0F701818734C080917A
:101D40007003813281F58091E800877F8093E800FD
:101D500066DC8091720390917303882736E0969534
:101D600087953A95E1F7F701958784871CC08091A4
:101D70007003813AC1F48091E800877F8093E80086
:101D80008091E80080FFFCCFF701848595859695CA
:101D90008795969587958093F1008091E8008E77DE
:101DA0008093E8003CDC0FB6F894DEBE0FBECDBEDB
:101DB0000F900F900F90DF91CF911F910F91FF9097
:101DC000EF90DF90CF90BF90AF909F908F907F90DB
:101DD0006F900895FC01399627E0DF011D922A9546
:101DE000E9F721E0FC01218724EF31E035872487E2
:101DF00023E0248361E00196C9CB4F925F926F92FA
:101E00007F928F929F92AF92BF92CF92DF92EF928A
:101E1000FF920F931F93CF93DF9300D01F92CDB704
:101E2000DEB77C01ADB6BEB680916F03843009F099
:101E30008EC08091E4009091E500F7012285338502
:101E40002817390709F483C081818F708093E900D6
:101E50008091E80085FF7BC08DB69EB6408550E03E
:101E60008DB79EB7841B950B0FB6F8949EBF0FBE1F
:101E70008DBFEDB7FEB731966F011B821A821982B2
:101E800060E070E0CF01A9D08E010F5F1F4F960177
:101E900040E0BE016D5F7F4FC7010E949E01482E4A
:101EA000F70184859585892B51F091E080E02685A6
:101EB0003785232B09F090E0092F182F02C000E08E
:101EC00010E0F701668077806114710489F0498120
:101ED0005A81B301C6016BD055245394892B09F460
:101EE000512CF701408550E0B601C3016DD001C00F
:101EF000512C89819A81892BF1F0411004C0511035
:101F000002C0012BC1F0F7018485958597878687EC
:101F100081818F708093E9008B8181118093F10022
:101F200069817A8140E050E0C601C3D98091E80020
:101F30008E778093E8008091E4009091E500F701AE
:101F4000938782870FB6F8949EBE0FBE8DBE0FB6E4
:101F5000F894BEBE0FBEADBE0F900F900F90DF91F4
:101F6000CF911F910F91FF90EF90DF90CF90BF9096
:101F7000AF909F908F907F906F905F904F9008955B
:101F80000024552704C0080E591F880F991F009779
:101F900029F076956795B8F37105B9F7802D952FDF
:101FA0000895EE0FFF1F0590F491E02D0994FB01B9
:101FB000DC0104C08D910190801921F44150504002
:101FC000C8F7881B990B0895FB01DC0102C0019042
:101FD0000D9241505040D8F70895DC0101C06D9337
:101FE00041505040E0F70895DC01CB01FC01F99924
:101FF000FECF06C0F2BDE1BDF89A319600B40D9255
:1020000041505040B8F70895F999FECF92BD81BD77
:10201000F89A992780B50895DC01A40FB51F4150A7
:10202000504040F0CB01840F951F2E9105D04150B8
:102030005040D8F70895262FF999FECF92BD81BD63
:10204000F89A019700B4021639F01FBA20BD0FB6F6
:0E205000F894FA9AF99A0FBE0895F894FFCF0B
:10205E000282190000015601190000000000000064
:10206E000183080000016F0108000000000000005D
:10207E000081080000017701080000000000000048
:10208E0050020200182520BE58027A019A0126013C
:10209E003F0158011003F401AC021003F401AC022D
:0620AE00302E362E360034
:00000001FF
